
D:\STM32\Program\1.11_Odchudzanie\um0427\FWLib\project\RIDE\STM3210E-EVAL\GRAPH.o:     file format elf32-littlearm
D:\STM32\Program\1.11_Odchudzanie\um0427\FWLib\project\RIDE\STM3210E-EVAL\GRAPH.o

Disassembly of section .text.GRAPH_ReadByteFromROMMemory:

00000000 <GRAPH_ReadByteFromROMMemory>:
GRAPH_ReadByteFromROMMemory():
D:\STM32\Program\1.11_Odchudzanie\um0427\FWLib\project/GRAPH.c:30
   0:	4b05      	ldr	r3, [pc, #20]	(18 <GRAPH_ReadByteFromROMMemory+0x18>)
   2:	781b      	ldrb	r3, [r3, #0]
   4:	2bff      	cmp	r3, #255
   6:	d103      	bne.n	10 <GRAPH_ReadByteFromROMMemory+0x10>
D:\STM32\Program\1.11_Odchudzanie\um0427\FWLib\project/GRAPH.c:31
   8:	7803      	ldrb	r3, [r0, #0]
   a:	43db      	mvns	r3, r3
   c:	b2d8      	uxtb	r0, r3
   e:	e001      	b.n	14 <GRAPH_ReadByteFromROMMemory+0x14>
D:\STM32\Program\1.11_Odchudzanie\um0427\FWLib\project/GRAPH.c:33
  10:	7803      	ldrb	r3, [r0, #0]
  12:	4618      	mov	r0, r3
D:\STM32\Program\1.11_Odchudzanie\um0427\FWLib\project/GRAPH.c:35
  14:	4770      	bx	lr
  16:	46c0      	nop			(mov r8, r8)
  18:	00000000 	.word	0x00000000
Disassembly of section .text.GRAPH_BlackWhite:

00000000 <GRAPH_BlackWhite>:
GRAPH_BlackWhite():
D:\STM32\Program\1.11_Odchudzanie\um0427\FWLib\project/GRAPH.c:98
   0:	4b02      	ldr	r3, [pc, #8]	(c <GRAPH_BlackWhite+0xc>)
   2:	f04f 32ff 	mov.w	r2, #4294967295	; 0xffffffff
   6:	701a      	strb	r2, [r3, #0]
D:\STM32\Program\1.11_Odchudzanie\um0427\FWLib\project/GRAPH.c:99
   8:	4770      	bx	lr
   a:	46c0      	nop			(mov r8, r8)
   c:	00000000 	.word	0x00000000
Disassembly of section .text.GRAPH_WhiteBlack:

00000000 <GRAPH_WhiteBlack>:
GRAPH_WhiteBlack():
D:\STM32\Program\1.11_Odchudzanie\um0427\FWLib\project/GRAPH.c:101
   0:	4b01      	ldr	r3, [pc, #4]	(8 <GRAPH_WhiteBlack+0x8>)
   2:	2200      	movs	r2, #0
   4:	701a      	strb	r2, [r3, #0]
D:\STM32\Program\1.11_Odchudzanie\um0427\FWLib\project/GRAPH.c:102
   6:	4770      	bx	lr
   8:	00000000 	.word	0x00000000
Disassembly of section .text.GRAPH_ClearScreen:

00000000 <GRAPH_ClearScreen>:
GRAPH_ClearScreen():
D:\STM32\Program\1.11_Odchudzanie\um0427\FWLib\project/GRAPH.c:46
   0:	b510      	push	{r4, lr}
D:\STM32\Program\1.11_Odchudzanie\um0427\FWLib\project/GRAPH.c:47
   2:	f7ff fffe 	bl	0 <GLCD_Clear_Text>
D:\STM32\Program\1.11_Odchudzanie\um0427\FWLib\project/GRAPH.c:48
   6:	f7ff fffe 	bl	0 <GLCD_Clear_CG>
D:\STM32\Program\1.11_Odchudzanie\um0427\FWLib\project/GRAPH.c:49
   a:	f7ff fffe 	bl	0 <GLCD_Clear_Graphic>
D:\STM32\Program\1.11_Odchudzanie\um0427\FWLib\project/GRAPH.c:50
   e:	bd10      	pop	{r4, pc}
Disassembly of section .text.GRAPH_TextGoTo:

00000000 <GRAPH_TextGoTo>:
GRAPH_TextGoTo():
D:\STM32\Program\1.11_Odchudzanie\um0427\FWLib\project/GRAPH.c:39
   0:	4b03      	ldr	r3, [pc, #12]	(10 <GRAPH_TextGoTo+0x10>)
D:\STM32\Program\1.11_Odchudzanie\um0427\FWLib\project/GRAPH.c:38
   2:	b510      	push	{r4, lr}
D:\STM32\Program\1.11_Odchudzanie\um0427\FWLib\project/GRAPH.c:39
   4:	7018      	strb	r0, [r3, #0]
D:\STM32\Program\1.11_Odchudzanie\um0427\FWLib\project/GRAPH.c:40
   6:	7059      	strb	r1, [r3, #1]
D:\STM32\Program\1.11_Odchudzanie\um0427\FWLib\project/GRAPH.c:42
   8:	f7ff fffe 	bl	0 <GLCD_Text_GoTo>
D:\STM32\Program\1.11_Odchudzanie\um0427\FWLib\project/GRAPH.c:43
   c:	bd10      	pop	{r4, pc}
   e:	46c0      	nop			(mov r8, r8)
  10:	00000000 	.word	0x00000000
Disassembly of section .text.GRAPH_SetPixel:

00000000 <GRAPH_SetPixel>:
GRAPH_SetPixel():
D:\STM32\Program\1.11_Odchudzanie\um0427\FWLib\project/GRAPH.c:24
   0:	b510      	push	{r4, lr}
D:\STM32\Program\1.11_Odchudzanie\um0427\FWLib\project/GRAPH.c:25
   2:	f7ff fffe 	bl	0 <GLCD_SetPixel>
D:\STM32\Program\1.11_Odchudzanie\um0427\FWLib\project/GRAPH.c:26
   6:	bd10      	pop	{r4, pc}
Disassembly of section .text.GRAPH_SquareRotated:

00000000 <GRAPH_SquareRotated>:
GRAPH_SquareRotated():
D:\STM32\Program\1.11_Odchudzanie\um0427\FWLib\project/GRAPH.c:255
   0:	e92d 4ff0 	stmdb	sp!, {r4, r5, r6, r7, r8, r9, sl, fp, lr}
   4:	b08f      	sub	sp, #60
   6:	9207      	str	r2, [sp, #28]
   8:	f99d 206c 	ldrsb.w	r2, [sp, #108]
   c:	9306      	str	r3, [sp, #24]
   e:	9009      	str	r0, [sp, #36]
  10:	9108      	str	r1, [sp, #32]
  12:	9205      	str	r2, [sp, #20]
D:\STM32\Program\1.11_Odchudzanie\um0427\FWLib\project/GRAPH.c:259
  14:	9b07      	ldr	r3, [sp, #28]
  16:	e08e      	b.n	136 <GRAPH_SquareRotated+0x136>
D:\STM32\Program\1.11_Odchudzanie\um0427\FWLib\project/GRAPH.c:262
  18:	981a      	ldr	r0, [sp, #104]
  1a:	f7ff fffe 	bl	0 <__aeabi_f2d>
  1e:	4604      	mov	r4, r0
  20:	460d      	mov	r5, r1
  22:	f7ff fffe 	bl	0 <cos>
  26:	e9cd 010a 	strd	r0, r1, [sp, #40]
  2a:	4638      	mov	r0, r7
  2c:	f7ff fffe 	bl	0 <__aeabi_ui2f>
  30:	f7ff fffe 	bl	0 <__aeabi_f2d>
  34:	e9dd 230a 	ldrd	r2, r3, [sp, #40]
  38:	f7ff fffe 	bl	0 <__aeabi_dmul>
  3c:	e9cd 0102 	strd	r0, r1, [sp, #8]
  40:	9806      	ldr	r0, [sp, #24]
  42:	f7ff fffe 	bl	0 <__aeabi_i2f>
  46:	f7ff fffe 	bl	0 <__aeabi_f2d>
  4a:	4682      	mov	sl, r0
  4c:	468b      	mov	fp, r1
  4e:	4620      	mov	r0, r4
  50:	4629      	mov	r1, r5
  52:	f7ff fffe 	bl	0 <sin>
  56:	4680      	mov	r8, r0
  58:	4689      	mov	r9, r1
  5a:	4650      	mov	r0, sl
  5c:	4659      	mov	r1, fp
  5e:	4642      	mov	r2, r8
  60:	464b      	mov	r3, r9
  62:	f7ff fffe 	bl	0 <__aeabi_dmul>
  66:	460b      	mov	r3, r1
  68:	4602      	mov	r2, r0
  6a:	e9dd 0102 	ldrd	r0, r1, [sp, #8]
  6e:	f7ff fffe 	bl	0 <__aeabi_dsub>
  72:	f7ff fffe 	bl	0 <__aeabi_d2f>
  76:	4604      	mov	r4, r0
D:\STM32\Program\1.11_Odchudzanie\um0427\FWLib\project/GRAPH.c:266
  78:	f7ff fffe 	bl	0 <__aeabi_f2iz>
  7c:	9a09      	ldr	r2, [sp, #36]
  7e:	1886      	adds	r6, r0, r2
  80:	4620      	mov	r0, r4
  82:	f7ff fffe 	bl	0 <__aeabi_f2d>
  86:	4642      	mov	r2, r8
  88:	464b      	mov	r3, r9
  8a:	f7ff fffe 	bl	0 <__aeabi_dmul>
  8e:	e9dd 230a 	ldrd	r2, r3, [sp, #40]
  92:	4604      	mov	r4, r0
  94:	460d      	mov	r5, r1
  96:	4650      	mov	r0, sl
  98:	4659      	mov	r1, fp
  9a:	f7ff fffe 	bl	0 <__aeabi_dmul>
  9e:	4602      	mov	r2, r0
  a0:	460b      	mov	r3, r1
  a2:	4620      	mov	r0, r4
  a4:	4629      	mov	r1, r5
  a6:	f7ff fffe 	bl	0 <__aeabi_dadd>
  aa:	f7ff fffe 	bl	0 <__aeabi_d2f>
  ae:	f7ff fffe 	bl	0 <__aeabi_f2iz>
  b2:	9b08      	ldr	r3, [sp, #32]
  b4:	b2f6      	uxtb	r6, r6
  b6:	18c1      	adds	r1, r0, r3
  b8:	9a05      	ldr	r2, [sp, #20]
  ba:	4630      	mov	r0, r6
  bc:	b2c9      	uxtb	r1, r1
  be:	f7ff fffe 	bl	0 <GRAPH_SquareRotated>
D:\STM32\Program\1.11_Odchudzanie\um0427\FWLib\project/GRAPH.c:269
  c2:	9819      	ldr	r0, [sp, #100]
  c4:	f7ff fffe 	bl	0 <__aeabi_i2f>
  c8:	f7ff fffe 	bl	0 <__aeabi_f2d>
  cc:	4642      	mov	r2, r8
  ce:	464b      	mov	r3, r9
  d0:	4682      	mov	sl, r0
  d2:	468b      	mov	fp, r1
  d4:	f7ff fffe 	bl	0 <__aeabi_dmul>
  d8:	460b      	mov	r3, r1
  da:	4602      	mov	r2, r0
  dc:	e9dd 0102 	ldrd	r0, r1, [sp, #8]
  e0:	f7ff fffe 	bl	0 <__aeabi_dsub>
  e4:	f7ff fffe 	bl	0 <__aeabi_d2f>
  e8:	4604      	mov	r4, r0
D:\STM32\Program\1.11_Odchudzanie\um0427\FWLib\project/GRAPH.c:273
  ea:	f7ff fffe 	bl	0 <__aeabi_f2iz>
  ee:	9a09      	ldr	r2, [sp, #36]
  f0:	1886      	adds	r6, r0, r2
  f2:	4620      	mov	r0, r4
  f4:	f7ff fffe 	bl	0 <__aeabi_f2d>
  f8:	4642      	mov	r2, r8
  fa:	464b      	mov	r3, r9
  fc:	f7ff fffe 	bl	0 <__aeabi_dmul>
 100:	e9dd 230a 	ldrd	r2, r3, [sp, #40]
 104:	4604      	mov	r4, r0
 106:	460d      	mov	r5, r1
 108:	4650      	mov	r0, sl
 10a:	4659      	mov	r1, fp
 10c:	f7ff fffe 	bl	0 <__aeabi_dmul>
 110:	4602      	mov	r2, r0
 112:	460b      	mov	r3, r1
 114:	4620      	mov	r0, r4
 116:	4629      	mov	r1, r5
 118:	f7ff fffe 	bl	0 <__aeabi_dadd>
 11c:	f7ff fffe 	bl	0 <__aeabi_d2f>
 120:	f7ff fffe 	bl	0 <__aeabi_f2iz>
 124:	9b08      	ldr	r3, [sp, #32]
 126:	b2f6      	uxtb	r6, r6
 128:	18c1      	adds	r1, r0, r3
 12a:	b2c9      	uxtb	r1, r1
 12c:	4630      	mov	r0, r6
 12e:	9a05      	ldr	r2, [sp, #20]
 130:	f7ff fffe 	bl	0 <GRAPH_SquareRotated>
D:\STM32\Program\1.11_Odchudzanie\um0427\FWLib\project/GRAPH.c:259
 134:	1c7b      	adds	r3, r7, #1
 136:	9a18      	ldr	r2, [sp, #96]
 138:	b2df      	uxtb	r7, r3
 13a:	1c53      	adds	r3, r2, #1
 13c:	429f      	cmp	r7, r3
 13e:	f6ff af6b 	blt.w	18 <GRAPH_SquareRotated+0x18>
D:\STM32\Program\1.11_Odchudzanie\um0427\FWLib\project/GRAPH.c:276
 142:	9b06      	ldr	r3, [sp, #24]
 144:	e07e      	b.n	244 <GRAPH_SquareRotated+0x244>
D:\STM32\Program\1.11_Odchudzanie\um0427\FWLib\project/GRAPH.c:279
 146:	981a      	ldr	r0, [sp, #104]
 148:	f7ff fffe 	bl	0 <__aeabi_f2d>
 14c:	4604      	mov	r4, r0
 14e:	460d      	mov	r5, r1
 150:	f7ff fffe 	bl	0 <cos>
 154:	4680      	mov	r8, r0
 156:	980d      	ldr	r0, [sp, #52]
 158:	4689      	mov	r9, r1
 15a:	f7ff fffe 	bl	0 <__aeabi_ui2f>
 15e:	f7ff fffe 	bl	0 <__aeabi_f2d>
 162:	4682      	mov	sl, r0
 164:	468b      	mov	fp, r1
 166:	4620      	mov	r0, r4
 168:	4629      	mov	r1, r5
 16a:	f7ff fffe 	bl	0 <sin>
 16e:	4606      	mov	r6, r0
 170:	460f      	mov	r7, r1
 172:	4632      	mov	r2, r6
 174:	463b      	mov	r3, r7
 176:	4650      	mov	r0, sl
 178:	4659      	mov	r1, fp
 17a:	f7ff fffe 	bl	0 <__aeabi_dmul>
 17e:	e9cd 0100 	strd	r0, r1, [sp]
 182:	9807      	ldr	r0, [sp, #28]
 184:	f7ff fffe 	bl	0 <__aeabi_i2f>
 188:	f7ff fffe 	bl	0 <__aeabi_f2d>
 18c:	4642      	mov	r2, r8
 18e:	464b      	mov	r3, r9
 190:	f7ff fffe 	bl	0 <__aeabi_dmul>
 194:	e9dd 2300 	ldrd	r2, r3, [sp]
 198:	f7ff fffe 	bl	0 <__aeabi_dsub>
 19c:	f7ff fffe 	bl	0 <__aeabi_d2f>
D:\STM32\Program\1.11_Odchudzanie\um0427\FWLib\project/GRAPH.c:280
 1a0:	464b      	mov	r3, r9
D:\STM32\Program\1.11_Odchudzanie\um0427\FWLib\project/GRAPH.c:279
 1a2:	4605      	mov	r5, r0
D:\STM32\Program\1.11_Odchudzanie\um0427\FWLib\project/GRAPH.c:280
 1a4:	4642      	mov	r2, r8
 1a6:	4650      	mov	r0, sl
 1a8:	4659      	mov	r1, fp
 1aa:	f7ff fffe 	bl	0 <__aeabi_dmul>
 1ae:	4682      	mov	sl, r0
D:\STM32\Program\1.11_Odchudzanie\um0427\FWLib\project/GRAPH.c:283
 1b0:	4628      	mov	r0, r5
D:\STM32\Program\1.11_Odchudzanie\um0427\FWLib\project/GRAPH.c:280
 1b2:	468b      	mov	fp, r1
D:\STM32\Program\1.11_Odchudzanie\um0427\FWLib\project/GRAPH.c:283
 1b4:	f7ff fffe 	bl	0 <__aeabi_f2iz>
 1b8:	9a09      	ldr	r2, [sp, #36]
 1ba:	1884      	adds	r4, r0, r2
 1bc:	4628      	mov	r0, r5
 1be:	f7ff fffe 	bl	0 <__aeabi_f2d>
 1c2:	4632      	mov	r2, r6
 1c4:	463b      	mov	r3, r7
 1c6:	f7ff fffe 	bl	0 <__aeabi_dmul>
 1ca:	4652      	mov	r2, sl
 1cc:	465b      	mov	r3, fp
 1ce:	f7ff fffe 	bl	0 <__aeabi_dadd>
 1d2:	f7ff fffe 	bl	0 <__aeabi_d2f>
 1d6:	f7ff fffe 	bl	0 <__aeabi_f2iz>
 1da:	9b08      	ldr	r3, [sp, #32]
 1dc:	b2e4      	uxtb	r4, r4
 1de:	18c1      	adds	r1, r0, r3
 1e0:	9a05      	ldr	r2, [sp, #20]
 1e2:	4620      	mov	r0, r4
 1e4:	b2c9      	uxtb	r1, r1
 1e6:	f7ff fffe 	bl	0 <GRAPH_SquareRotated>
D:\STM32\Program\1.11_Odchudzanie\um0427\FWLib\project/GRAPH.c:286
 1ea:	9818      	ldr	r0, [sp, #96]
 1ec:	f7ff fffe 	bl	0 <__aeabi_i2f>
 1f0:	f7ff fffe 	bl	0 <__aeabi_f2d>
 1f4:	4642      	mov	r2, r8
 1f6:	464b      	mov	r3, r9
 1f8:	f7ff fffe 	bl	0 <__aeabi_dmul>
 1fc:	e9dd 2300 	ldrd	r2, r3, [sp]
 200:	f7ff fffe 	bl	0 <__aeabi_dsub>
 204:	f7ff fffe 	bl	0 <__aeabi_d2f>
 208:	4605      	mov	r5, r0
D:\STM32\Program\1.11_Odchudzanie\um0427\FWLib\project/GRAPH.c:290
 20a:	f7ff fffe 	bl	0 <__aeabi_f2iz>
 20e:	9a09      	ldr	r2, [sp, #36]
 210:	1884      	adds	r4, r0, r2
 212:	4628      	mov	r0, r5
 214:	f7ff fffe 	bl	0 <__aeabi_f2d>
 218:	4632      	mov	r2, r6
 21a:	463b      	mov	r3, r7
 21c:	f7ff fffe 	bl	0 <__aeabi_dmul>
 220:	4652      	mov	r2, sl
 222:	465b      	mov	r3, fp
 224:	f7ff fffe 	bl	0 <__aeabi_dadd>
 228:	f7ff fffe 	bl	0 <__aeabi_d2f>
 22c:	f7ff fffe 	bl	0 <__aeabi_f2iz>
 230:	9b08      	ldr	r3, [sp, #32]
 232:	b2e4      	uxtb	r4, r4
 234:	18c1      	adds	r1, r0, r3
 236:	9a05      	ldr	r2, [sp, #20]
 238:	4620      	mov	r0, r4
 23a:	b2c9      	uxtb	r1, r1
 23c:	f7ff fffe 	bl	0 <GRAPH_SquareRotated>
D:\STM32\Program\1.11_Odchudzanie\um0427\FWLib\project/GRAPH.c:276
 240:	9a0d      	ldr	r2, [sp, #52]
 242:	1c53      	adds	r3, r2, #1
 244:	b2db      	uxtb	r3, r3
 246:	9a19      	ldr	r2, [sp, #100]
 248:	930d      	str	r3, [sp, #52]
 24a:	1c53      	adds	r3, r2, #1
 24c:	9a0d      	ldr	r2, [sp, #52]
 24e:	429a      	cmp	r2, r3
 250:	f6ff af79 	blt.w	146 <GRAPH_SquareRotated+0x146>
D:\STM32\Program\1.11_Odchudzanie\um0427\FWLib\project/GRAPH.c:292
 254:	b00f      	add	sp, #60
 256:	e8bd 8ff0 	ldmia.w	sp!, {r4, r5, r6, r7, r8, r9, sl, fp, pc}
 25a:	46c0      	nop			(mov r8, r8)
Disassembly of section .text.GRAPH_Line:

00000000 <GRAPH_Line>:
GRAPH_Line():
D:\STM32\Program\1.11_Odchudzanie\um0427\FWLib\project/GRAPH.c:184
   0:	e92d 4ff0 	stmdb	sp!, {r4, r5, r6, r7, r8, r9, sl, fp, lr}
   4:	b085      	sub	sp, #20
   6:	9202      	str	r2, [sp, #8]
   8:	f99d 2038 	ldrsb.w	r2, [sp, #56]
   c:	9301      	str	r3, [sp, #4]
D:\STM32\Program\1.11_Odchudzanie\um0427\FWLib\project/GRAPH.c:189
   e:	9b02      	ldr	r3, [sp, #8]
D:\STM32\Program\1.11_Odchudzanie\um0427\FWLib\project/GRAPH.c:184
  10:	9200      	str	r2, [sp, #0]
D:\STM32\Program\1.11_Odchudzanie\um0427\FWLib\project/GRAPH.c:190
  12:	9a01      	ldr	r2, [sp, #4]
D:\STM32\Program\1.11_Odchudzanie\um0427\FWLib\project/GRAPH.c:189
  14:	ebc0 0603 	rsb	r6, r0, r3
D:\STM32\Program\1.11_Odchudzanie\um0427\FWLib\project/GRAPH.c:190
  18:	1a55      	subs	r5, r2, r1
D:\STM32\Program\1.11_Odchudzanie\um0427\FWLib\project/GRAPH.c:201
  1a:	2e00      	cmp	r6, #0
D:\STM32\Program\1.11_Odchudzanie\um0427\FWLib\project/GRAPH.c:184
  1c:	4680      	mov	r8, r0
  1e:	460f      	mov	r7, r1
D:\STM32\Program\1.11_Odchudzanie\um0427\FWLib\project/GRAPH.c:192
  20:	ea4f 0a46 	mov.w	sl, r6, lsl #1
D:\STM32\Program\1.11_Odchudzanie\um0427\FWLib\project/GRAPH.c:193
  24:	ea4f 0945 	mov.w	r9, r5, lsl #1
D:\STM32\Program\1.11_Odchudzanie\um0427\FWLib\project/GRAPH.c:201
  28:	db02      	blt.n	30 <GRAPH_Line+0x30>
  2a:	2301      	movs	r3, #1
  2c:	9303      	str	r3, [sp, #12]
  2e:	e005      	b.n	3c <GRAPH_Line+0x3c>
D:\STM32\Program\1.11_Odchudzanie\um0427\FWLib\project/GRAPH.c:205
  30:	f04f 32ff 	mov.w	r2, #4294967295	; 0xffffffff
D:\STM32\Program\1.11_Odchudzanie\um0427\FWLib\project/GRAPH.c:204
  34:	4276      	negs	r6, r6
D:\STM32\Program\1.11_Odchudzanie\um0427\FWLib\project/GRAPH.c:205
  36:	f1ca 0a00 	rsb	sl, sl, #0	; 0x0
  3a:	9203      	str	r2, [sp, #12]
D:\STM32\Program\1.11_Odchudzanie\um0427\FWLib\project/GRAPH.c:208
  3c:	2d00      	cmp	r5, #0
  3e:	db02      	blt.n	46 <GRAPH_Line+0x46>
  40:	f04f 0b01 	mov.w	fp, #1	; 0x1
  44:	e004      	b.n	50 <GRAPH_Line+0x50>
D:\STM32\Program\1.11_Odchudzanie\um0427\FWLib\project/GRAPH.c:211
  46:	426d      	negs	r5, r5
D:\STM32\Program\1.11_Odchudzanie\um0427\FWLib\project/GRAPH.c:212
  48:	f1c9 0900 	rsb	r9, r9, #0	; 0x0
  4c:	f04f 3bff 	mov.w	fp, #4294967295	; 0xffffffff
D:\STM32\Program\1.11_Odchudzanie\um0427\FWLib\project/GRAPH.c:215
  50:	fa5f f088 	uxtb.w	r0, r8
  54:	b2f9      	uxtb	r1, r7
  56:	9a00      	ldr	r2, [sp, #0]
  58:	f7ff fffe 	bl	0 <GRAPH_Line>
D:\STM32\Program\1.11_Odchudzanie\um0427\FWLib\project/GRAPH.c:217
  5c:	b90e      	cbnz	r6, 62 <GRAPH_Line+0x62>
  5e:	2d00      	cmp	r5, #0
  60:	d02f      	beq.n	c2 <GRAPH_Line+0xc2>
D:\STM32\Program\1.11_Odchudzanie\um0427\FWLib\project/GRAPH.c:220
  62:	42b5      	cmp	r5, r6
  64:	dc17      	bgt.n	96 <GRAPH_Line+0x96>
  66:	9b03      	ldr	r3, [sp, #12]
  68:	463d      	mov	r5, r7
  6a:	eb03 0408 	add.w	r4, r3, r8
  6e:	2700      	movs	r7, #0
D:\STM32\Program\1.11_Odchudzanie\um0427\FWLib\project/GRAPH.c:226
  70:	444f      	add	r7, r9
D:\STM32\Program\1.11_Odchudzanie\um0427\FWLib\project/GRAPH.c:227
  72:	42b7      	cmp	r7, r6
D:\STM32\Program\1.11_Odchudzanie\um0427\FWLib\project/GRAPH.c:229
  74:	bfc8      	it	gt
  76:	445d      	addgt	r5, fp
D:\STM32\Program\1.11_Odchudzanie\um0427\FWLib\project/GRAPH.c:232
  78:	b2e0      	uxtb	r0, r4
  7a:	9a00      	ldr	r2, [sp, #0]
  7c:	b2e9      	uxtb	r1, r5
D:\STM32\Program\1.11_Odchudzanie\um0427\FWLib\project/GRAPH.c:230
  7e:	bfc8      	it	gt
  80:	ebca 0707 	rsbgt	r7, sl, r7
D:\STM32\Program\1.11_Odchudzanie\um0427\FWLib\project/GRAPH.c:232
  84:	f7ff fffe 	bl	0 <GRAPH_Line>
  88:	9a03      	ldr	r2, [sp, #12]
  8a:	18a4      	adds	r4, r4, r2
D:\STM32\Program\1.11_Odchudzanie\um0427\FWLib\project/GRAPH.c:233
  8c:	1aa3      	subs	r3, r4, r2
  8e:	9a02      	ldr	r2, [sp, #8]
  90:	4293      	cmp	r3, r2
  92:	d1ed      	bne.n	70 <GRAPH_Line+0x70>
  94:	e015      	b.n	c2 <GRAPH_Line+0xc2>
  96:	eb0b 0407 	add.w	r4, fp, r7
  9a:	4646      	mov	r6, r8
  9c:	2700      	movs	r7, #0
D:\STM32\Program\1.11_Odchudzanie\um0427\FWLib\project/GRAPH.c:241
  9e:	4457      	add	r7, sl
D:\STM32\Program\1.11_Odchudzanie\um0427\FWLib\project/GRAPH.c:242
  a0:	42af      	cmp	r7, r5
  a2:	dd03      	ble.n	ac <GRAPH_Line+0xac>
D:\STM32\Program\1.11_Odchudzanie\um0427\FWLib\project/GRAPH.c:244
  a4:	9b03      	ldr	r3, [sp, #12]
D:\STM32\Program\1.11_Odchudzanie\um0427\FWLib\project/GRAPH.c:245
  a6:	ebc9 0707 	rsb	r7, r9, r7
D:\STM32\Program\1.11_Odchudzanie\um0427\FWLib\project/GRAPH.c:244
  aa:	18f6      	adds	r6, r6, r3
D:\STM32\Program\1.11_Odchudzanie\um0427\FWLib\project/GRAPH.c:247
  ac:	b2e1      	uxtb	r1, r4
  ae:	9a00      	ldr	r2, [sp, #0]
  b0:	b2f0      	uxtb	r0, r6
  b2:	f7ff fffe 	bl	0 <GRAPH_Line>
  b6:	445c      	add	r4, fp
D:\STM32\Program\1.11_Odchudzanie\um0427\FWLib\project/GRAPH.c:248
  b8:	9a01      	ldr	r2, [sp, #4]
  ba:	ebcb 0304 	rsb	r3, fp, r4
  be:	4293      	cmp	r3, r2
  c0:	d1ed      	bne.n	9e <GRAPH_Line+0x9e>
D:\STM32\Program\1.11_Odchudzanie\um0427\FWLib\project/GRAPH.c:251
  c2:	b005      	add	sp, #20
  c4:	e8bd 8ff0 	ldmia.w	sp!, {r4, r5, r6, r7, r8, r9, sl, fp, pc}
Disassembly of section .text.GRAPH_TriangleFill:

00000000 <GRAPH_TriangleFill>:
GRAPH_TriangleFill():
D:\STM32\Program\1.11_Odchudzanie\um0427\FWLib\project/GRAPH.c:366
   0:	e92d 4ff0 	stmdb	sp!, {r4, r5, r6, r7, r8, r9, sl, fp, lr}
   4:	b087      	sub	sp, #28
   6:	4605      	mov	r5, r0
   8:	460f      	mov	r7, r1
   a:	9203      	str	r2, [sp, #12]
   c:	4604      	mov	r4, r0
   e:	f04f 0e00 	mov.w	lr, #0	; 0x0
D:\STM32\Program\1.11_Odchudzanie\um0427\FWLib\project/GRAPH.c:378
  12:	e00f      	b.n	34 <GRAPH_TriangleFill+0x34>
D:\STM32\Program\1.11_Odchudzanie\um0427\FWLib\project/GRAPH.c:379
  14:	6866      	ldr	r6, [r4, #4]
  16:	68e3      	ldr	r3, [r4, #12]
  18:	429e      	cmp	r6, r3
  1a:	da08      	bge.n	2e <GRAPH_TriangleFill+0x2e>
D:\STM32\Program\1.11_Odchudzanie\um0427\FWLib\project/GRAPH.c:381
  1c:	f104 0308 	add.w	r3, r4, #8	; 0x8
  20:	e893 0003 	ldmia.w	r3, {r0, r1}
D:\STM32\Program\1.11_Odchudzanie\um0427\FWLib\project/GRAPH.c:380
  24:	6822      	ldr	r2, [r4, #0]
D:\STM32\Program\1.11_Odchudzanie\um0427\FWLib\project/GRAPH.c:381
  26:	e884 0003 	stmia.w	r4, {r0, r1}
D:\STM32\Program\1.11_Odchudzanie\um0427\FWLib\project/GRAPH.c:382
  2a:	60e6      	str	r6, [r4, #12]
  2c:	60a2      	str	r2, [r4, #8]
D:\STM32\Program\1.11_Odchudzanie\um0427\FWLib\project/GRAPH.c:378
  2e:	f10e 0e01 	add.w	lr, lr, #1	; 0x1
  32:	3408      	adds	r4, #8
  34:	1e7b      	subs	r3, r7, #1
  36:	459e      	cmp	lr, r3
  38:	dbec      	blt.n	14 <GRAPH_TriangleFill+0x14>
D:\STM32\Program\1.11_Odchudzanie\um0427\FWLib\project/GRAPH.c:386
  3a:	f8d5 800c 	ldr.w	r8, [r5, #12]
D:\STM32\Program\1.11_Odchudzanie\um0427\FWLib\project/GRAPH.c:387
  3e:	696e      	ldr	r6, [r5, #20]
D:\STM32\Program\1.11_Odchudzanie\um0427\FWLib\project/GRAPH.c:385
  40:	f8d5 a000 	ldr.w	sl, [r5]
  44:	f8d5 b004 	ldr.w	fp, [r5, #4]
D:\STM32\Program\1.11_Odchudzanie\um0427\FWLib\project/GRAPH.c:386
  48:	f8d5 9008 	ldr.w	r9, [r5, #8]
D:\STM32\Program\1.11_Odchudzanie\um0427\FWLib\project/GRAPH.c:387
  4c:	692f      	ldr	r7, [r5, #16]
D:\STM32\Program\1.11_Odchudzanie\um0427\FWLib\project/GRAPH.c:390
  4e:	ebc6 0508 	rsb	r5, r6, r8
  52:	2d00      	cmp	r5, #0
  54:	dc02      	bgt.n	5c <GRAPH_TriangleFill+0x5c>
  56:	2200      	movs	r2, #0
  58:	9204      	str	r2, [sp, #16]
  5a:	e00c      	b.n	76 <GRAPH_TriangleFill+0x76>
  5c:	ebc7 0009 	rsb	r0, r7, r9
  60:	f7ff fffe 	bl	0 <__aeabi_i2f>
  64:	4604      	mov	r4, r0
  66:	4628      	mov	r0, r5
  68:	f7ff fffe 	bl	0 <__aeabi_i2f>
  6c:	4601      	mov	r1, r0
  6e:	4620      	mov	r0, r4
  70:	f7ff fffe 	bl	0 <__aeabi_fdiv>
  74:	9004      	str	r0, [sp, #16]
D:\STM32\Program\1.11_Odchudzanie\um0427\FWLib\project/GRAPH.c:391
  76:	ebc6 050b 	rsb	r5, r6, fp
  7a:	2d00      	cmp	r5, #0
  7c:	dc02      	bgt.n	84 <GRAPH_TriangleFill+0x84>
  7e:	2300      	movs	r3, #0
  80:	9305      	str	r3, [sp, #20]
  82:	e00c      	b.n	9e <GRAPH_TriangleFill+0x9e>
  84:	ebc7 000a 	rsb	r0, r7, sl
  88:	f7ff fffe 	bl	0 <__aeabi_i2f>
  8c:	4604      	mov	r4, r0
  8e:	4628      	mov	r0, r5
  90:	f7ff fffe 	bl	0 <__aeabi_i2f>
  94:	4601      	mov	r1, r0
  96:	4620      	mov	r0, r4
  98:	f7ff fffe 	bl	0 <__aeabi_fdiv>
  9c:	9005      	str	r0, [sp, #20]
D:\STM32\Program\1.11_Odchudzanie\um0427\FWLib\project/GRAPH.c:392
  9e:	ebc8 050b 	rsb	r5, r8, fp
  a2:	2d00      	cmp	r5, #0
  a4:	dc02      	bgt.n	ac <GRAPH_TriangleFill+0xac>
  a6:	f04f 0a00 	mov.w	sl, #0	; 0x0
  aa:	e00c      	b.n	c6 <GRAPH_TriangleFill+0xc6>
  ac:	ebc9 000a 	rsb	r0, r9, sl
  b0:	f7ff fffe 	bl	0 <__aeabi_i2f>
  b4:	4604      	mov	r4, r0
  b6:	4628      	mov	r0, r5
  b8:	f7ff fffe 	bl	0 <__aeabi_i2f>
  bc:	4601      	mov	r1, r0
  be:	4620      	mov	r0, r4
  c0:	f7ff fffe 	bl	0 <__aeabi_fdiv>
  c4:	4682      	mov	sl, r0
D:\STM32\Program\1.11_Odchudzanie\um0427\FWLib\project/GRAPH.c:396
  c6:	9804      	ldr	r0, [sp, #16]
  c8:	9905      	ldr	r1, [sp, #20]
  ca:	f7ff fffe 	bl	0 <__aeabi_fcmpgt>
  ce:	b918      	cbnz	r0, d8 <GRAPH_TriangleFill+0xd8>
  d0:	4635      	mov	r5, r6
  d2:	463c      	mov	r4, r7
  d4:	463e      	mov	r6, r7
  d6:	e05e      	b.n	196 <GRAPH_TriangleFill+0x196>
  d8:	4635      	mov	r5, r6
  da:	463c      	mov	r4, r7
  dc:	463e      	mov	r6, r7
  de:	e01b      	b.n	118 <GRAPH_TriangleFill+0x118>
D:\STM32\Program\1.11_Odchudzanie\um0427\FWLib\project/GRAPH.c:398
  e0:	9a03      	ldr	r2, [sp, #12]
  e2:	4629      	mov	r1, r5
  e4:	b253      	sxtb	r3, r2
  e6:	4620      	mov	r0, r4
  e8:	4632      	mov	r2, r6
  ea:	9300      	str	r3, [sp, #0]
  ec:	462b      	mov	r3, r5
  ee:	f7ff fffe 	bl	0 <GRAPH_TriangleFill>
D:\STM32\Program\1.11_Odchudzanie\um0427\FWLib\project/GRAPH.c:397
  f2:	4620      	mov	r0, r4
  f4:	f7ff fffe 	bl	0 <__aeabi_i2f>
  f8:	9905      	ldr	r1, [sp, #20]
  fa:	f7ff fffe 	bl	0 <__aeabi_fadd>
  fe:	f7ff fffe 	bl	0 <__aeabi_f2iz>
 102:	4604      	mov	r4, r0
 104:	4630      	mov	r0, r6
 106:	f7ff fffe 	bl	0 <__aeabi_i2f>
 10a:	9904      	ldr	r1, [sp, #16]
 10c:	f7ff fffe 	bl	0 <__aeabi_fadd>
 110:	f7ff fffe 	bl	0 <__aeabi_f2iz>
 114:	3501      	adds	r5, #1
 116:	4606      	mov	r6, r0
 118:	4545      	cmp	r5, r8
 11a:	dde1      	ble.n	e0 <GRAPH_TriangleFill+0xe0>
 11c:	464e      	mov	r6, r9
 11e:	e01b      	b.n	158 <GRAPH_TriangleFill+0x158>
D:\STM32\Program\1.11_Odchudzanie\um0427\FWLib\project/GRAPH.c:401
 120:	9a03      	ldr	r2, [sp, #12]
 122:	4629      	mov	r1, r5
 124:	b253      	sxtb	r3, r2
 126:	4620      	mov	r0, r4
 128:	4632      	mov	r2, r6
 12a:	9300      	str	r3, [sp, #0]
 12c:	462b      	mov	r3, r5
 12e:	f7ff fffe 	bl	0 <GRAPH_TriangleFill>
D:\STM32\Program\1.11_Odchudzanie\um0427\FWLib\project/GRAPH.c:400
 132:	4620      	mov	r0, r4
 134:	f7ff fffe 	bl	0 <__aeabi_i2f>
 138:	9905      	ldr	r1, [sp, #20]
 13a:	f7ff fffe 	bl	0 <__aeabi_fadd>
 13e:	f7ff fffe 	bl	0 <__aeabi_f2iz>
 142:	4604      	mov	r4, r0
 144:	4630      	mov	r0, r6
 146:	f7ff fffe 	bl	0 <__aeabi_i2f>
 14a:	4651      	mov	r1, sl
 14c:	f7ff fffe 	bl	0 <__aeabi_fadd>
 150:	f7ff fffe 	bl	0 <__aeabi_f2iz>
 154:	3501      	adds	r5, #1
 156:	4606      	mov	r6, r0
 158:	455d      	cmp	r5, fp
 15a:	dde1      	ble.n	120 <GRAPH_TriangleFill+0x120>
 15c:	e03e      	b.n	1dc <GRAPH_TriangleFill+0x1dc>
D:\STM32\Program\1.11_Odchudzanie\um0427\FWLib\project/GRAPH.c:404
 15e:	9a03      	ldr	r2, [sp, #12]
 160:	4629      	mov	r1, r5
 162:	b253      	sxtb	r3, r2
 164:	4630      	mov	r0, r6
 166:	4622      	mov	r2, r4
 168:	9300      	str	r3, [sp, #0]
 16a:	462b      	mov	r3, r5
 16c:	f7ff fffe 	bl	0 <GRAPH_TriangleFill>
D:\STM32\Program\1.11_Odchudzanie\um0427\FWLib\project/GRAPH.c:403
 170:	4630      	mov	r0, r6
 172:	f7ff fffe 	bl	0 <__aeabi_i2f>
 176:	9904      	ldr	r1, [sp, #16]
 178:	f7ff fffe 	bl	0 <__aeabi_fadd>
 17c:	f7ff fffe 	bl	0 <__aeabi_f2iz>
 180:	4606      	mov	r6, r0
 182:	4620      	mov	r0, r4
 184:	f7ff fffe 	bl	0 <__aeabi_i2f>
 188:	9905      	ldr	r1, [sp, #20]
 18a:	f7ff fffe 	bl	0 <__aeabi_fadd>
 18e:	f7ff fffe 	bl	0 <__aeabi_f2iz>
 192:	3501      	adds	r5, #1
 194:	4604      	mov	r4, r0
 196:	4545      	cmp	r5, r8
 198:	dde1      	ble.n	15e <GRAPH_TriangleFill+0x15e>
 19a:	4645      	mov	r5, r8
 19c:	464e      	mov	r6, r9
 19e:	e01b      	b.n	1d8 <GRAPH_TriangleFill+0x1d8>
D:\STM32\Program\1.11_Odchudzanie\um0427\FWLib\project/GRAPH.c:407
 1a0:	9a03      	ldr	r2, [sp, #12]
 1a2:	4629      	mov	r1, r5
 1a4:	b253      	sxtb	r3, r2
 1a6:	4630      	mov	r0, r6
 1a8:	4622      	mov	r2, r4
 1aa:	9300      	str	r3, [sp, #0]
 1ac:	462b      	mov	r3, r5
 1ae:	f7ff fffe 	bl	0 <GRAPH_TriangleFill>
D:\STM32\Program\1.11_Odchudzanie\um0427\FWLib\project/GRAPH.c:406
 1b2:	4630      	mov	r0, r6
 1b4:	f7ff fffe 	bl	0 <__aeabi_i2f>
 1b8:	4651      	mov	r1, sl
 1ba:	f7ff fffe 	bl	0 <__aeabi_fadd>
 1be:	f7ff fffe 	bl	0 <__aeabi_f2iz>
 1c2:	4606      	mov	r6, r0
 1c4:	4620      	mov	r0, r4
 1c6:	f7ff fffe 	bl	0 <__aeabi_i2f>
 1ca:	9905      	ldr	r1, [sp, #20]
 1cc:	f7ff fffe 	bl	0 <__aeabi_fadd>
 1d0:	f7ff fffe 	bl	0 <__aeabi_f2iz>
 1d4:	3501      	adds	r5, #1
 1d6:	4604      	mov	r4, r0
 1d8:	455d      	cmp	r5, fp
 1da:	dde1      	ble.n	1a0 <__aeabi_f2iz+0x1a0>
D:\STM32\Program\1.11_Odchudzanie\um0427\FWLib\project/GRAPH.c:410
 1dc:	b007      	add	sp, #28
 1de:	e8bd 8ff0 	ldmia.w	sp!, {r4, r5, r6, r7, r8, r9, sl, fp, pc}
 1e2:	46c0      	nop			(mov r8, r8)
Disassembly of section .text.GRAPH_Arrow:

00000000 <GRAPH_Arrow>:
GRAPH_Arrow():
D:\STM32\Program\1.11_Odchudzanie\um0427\FWLib\project/GRAPH.c:295
   0:	e92d 4f70 	stmdb	sp!, {r4, r5, r6, r8, r9, sl, fp, lr}
   4:	4606      	mov	r6, r0
   6:	b086      	sub	sp, #24
D:\STM32\Program\1.11_Odchudzanie\um0427\FWLib\project/GRAPH.c:318
   8:	4610      	mov	r0, r2
D:\STM32\Program\1.11_Odchudzanie\um0427\FWLib\project/GRAPH.c:295
   a:	461d      	mov	r5, r3
D:\STM32\Program\1.11_Odchudzanie\um0427\FWLib\project/GRAPH.c:314
   c:	9200      	str	r2, [sp, #0]
D:\STM32\Program\1.11_Odchudzanie\um0427\FWLib\project/GRAPH.c:315
   e:	9301      	str	r3, [sp, #4]
D:\STM32\Program\1.11_Odchudzanie\um0427\FWLib\project/GRAPH.c:295
  10:	4688      	mov	r8, r1
D:\STM32\Program\1.11_Odchudzanie\um0427\FWLib\project/GRAPH.c:318
  12:	f7ff fffe 	bl	0 <__aeabi_i2f>
  16:	4604      	mov	r4, r0
  18:	4630      	mov	r0, r6
  1a:	f7ff fffe 	bl	0 <__aeabi_i2f>
  1e:	4601      	mov	r1, r0
  20:	4620      	mov	r0, r4
  22:	f7ff fffe 	bl	0 <__aeabi_fsub>
  26:	4681      	mov	r9, r0
D:\STM32\Program\1.11_Odchudzanie\um0427\FWLib\project/GRAPH.c:319
  28:	4628      	mov	r0, r5
  2a:	f7ff fffe 	bl	0 <__aeabi_i2f>
  2e:	4604      	mov	r4, r0
  30:	4640      	mov	r0, r8
  32:	f7ff fffe 	bl	0 <__aeabi_i2f>
  36:	4601      	mov	r1, r0
  38:	4620      	mov	r0, r4
  3a:	f7ff fffe 	bl	0 <__aeabi_fsub>
D:\STM32\Program\1.11_Odchudzanie\um0427\FWLib\project/GRAPH.c:326
  3e:	4649      	mov	r1, r9
D:\STM32\Program\1.11_Odchudzanie\um0427\FWLib\project/GRAPH.c:319
  40:	4605      	mov	r5, r0
D:\STM32\Program\1.11_Odchudzanie\um0427\FWLib\project/GRAPH.c:322
  42:	f100 4b00 	add.w	fp, r0, #2147483648	; 0x80000000
D:\STM32\Program\1.11_Odchudzanie\um0427\FWLib\project/GRAPH.c:326
  46:	4648      	mov	r0, r9
  48:	f7ff fffe 	bl	0 <__aeabi_fmul>
  4c:	4629      	mov	r1, r5
  4e:	4604      	mov	r4, r0
  50:	4628      	mov	r0, r5
  52:	f7ff fffe 	bl	0 <__aeabi_fmul>
  56:	4601      	mov	r1, r0
  58:	4620      	mov	r0, r4
  5a:	f7ff fffe 	bl	0 <__aeabi_fadd>
  5e:	f7ff fffe 	bl	0 <__aeabi_f2d>
  62:	f7ff fffe 	bl	0 <sqrt>
  66:	f7ff fffe 	bl	0 <__aeabi_d2f>
  6a:	4604      	mov	r4, r0
D:\STM32\Program\1.11_Odchudzanie\um0427\FWLib\project/GRAPH.c:327
  6c:	4621      	mov	r1, r4
  6e:	f7ff fffe 	bl	0 <__aeabi_fadd>
  72:	f8df 80ec 	ldr.w	r8, [pc, #236]	; 160 <GRAPH_Arrow+0x160>
  76:	4601      	mov	r1, r0
  78:	4640      	mov	r0, r8
  7a:	f7ff fffe 	bl	0 <__aeabi_fdiv>
  7e:	4606      	mov	r6, r0
D:\STM32\Program\1.11_Odchudzanie\um0427\FWLib\project/GRAPH.c:328
  80:	4836      	ldr	r0, [pc, #216]	(15c <GRAPH_Arrow+0x15c>)
  82:	f7ff fffe 	bl	0 <tanf>
D:\STM32\Program\1.11_Odchudzanie\um0427\FWLib\project/GRAPH.c:331
  86:	f04f 517c 	mov.w	r1, #1056964608	; 0x3f000000
  8a:	f7ff fffe 	bl	0 <__aeabi_fmul>
  8e:	4601      	mov	r1, r0
  90:	f7ff fffe 	bl	0 <__aeabi_fadd>
  94:	4621      	mov	r1, r4
  96:	f7ff fffe 	bl	0 <__aeabi_fmul>
  9a:	4601      	mov	r1, r0
  9c:	4640      	mov	r0, r8
  9e:	f7ff fffe 	bl	0 <__aeabi_fdiv>
  a2:	f100 4800 	add.w	r8, r0, #2147483648	; 0x80000000
D:\STM32\Program\1.11_Odchudzanie\um0427\FWLib\project/GRAPH.c:332
  a6:	9801      	ldr	r0, [sp, #4]
  a8:	f7ff fffe 	bl	0 <__aeabi_i2f>
  ac:	4629      	mov	r1, r5
  ae:	4604      	mov	r4, r0
  b0:	4640      	mov	r0, r8
  b2:	f7ff fffe 	bl	0 <__aeabi_fmul>
  b6:	4601      	mov	r1, r0
  b8:	4620      	mov	r0, r4
  ba:	f7ff fffe 	bl	0 <__aeabi_fadd>
  be:	f7ff fffe 	bl	0 <__aeabi_f2iz>
  c2:	4682      	mov	sl, r0
D:\STM32\Program\1.11_Odchudzanie\um0427\FWLib\project/GRAPH.c:335
  c4:	9800      	ldr	r0, [sp, #0]
  c6:	f7ff fffe 	bl	0 <__aeabi_i2f>
  ca:	4649      	mov	r1, r9
  cc:	4604      	mov	r4, r0
  ce:	4640      	mov	r0, r8
  d0:	f7ff fffe 	bl	0 <__aeabi_fmul>
  d4:	4601      	mov	r1, r0
  d6:	4620      	mov	r0, r4
  d8:	f7ff fffe 	bl	0 <__aeabi_fadd>
  dc:	f7ff fffe 	bl	0 <__aeabi_f2iz>
  e0:	f7ff fffe 	bl	0 <__aeabi_i2f>
  e4:	4659      	mov	r1, fp
  e6:	4605      	mov	r5, r0
  e8:	4630      	mov	r0, r6
  ea:	f7ff fffe 	bl	0 <__aeabi_fmul>
  ee:	4601      	mov	r1, r0
  f0:	4628      	mov	r0, r5
  f2:	f7ff fffe 	bl	0 <__aeabi_fadd>
  f6:	f7ff fffe 	bl	0 <__aeabi_f2iz>
  fa:	9002      	str	r0, [sp, #8]
D:\STM32\Program\1.11_Odchudzanie\um0427\FWLib\project/GRAPH.c:336
  fc:	4650      	mov	r0, sl
  fe:	f7ff fffe 	bl	0 <__aeabi_i2f>
 102:	4649      	mov	r1, r9
 104:	4604      	mov	r4, r0
 106:	4630      	mov	r0, r6
 108:	f7ff fffe 	bl	0 <__aeabi_fmul>
 10c:	4601      	mov	r1, r0
 10e:	4620      	mov	r0, r4
 110:	f7ff fffe 	bl	0 <__aeabi_fadd>
 114:	f7ff fffe 	bl	0 <__aeabi_f2iz>
D:\STM32\Program\1.11_Odchudzanie\um0427\FWLib\project/GRAPH.c:337
 118:	f106 4600 	add.w	r6, r6, #2147483648	; 0x80000000
D:\STM32\Program\1.11_Odchudzanie\um0427\FWLib\project/GRAPH.c:336
 11c:	9003      	str	r0, [sp, #12]
D:\STM32\Program\1.11_Odchudzanie\um0427\FWLib\project/GRAPH.c:337
 11e:	4659      	mov	r1, fp
 120:	4630      	mov	r0, r6
 122:	f7ff fffe 	bl	0 <__aeabi_fmul>
 126:	4601      	mov	r1, r0
 128:	4628      	mov	r0, r5
 12a:	f7ff fffe 	bl	0 <__aeabi_fadd>
 12e:	f7ff fffe 	bl	0 <__aeabi_f2iz>
D:\STM32\Program\1.11_Odchudzanie\um0427\FWLib\project/GRAPH.c:338
 132:	4649      	mov	r1, r9
D:\STM32\Program\1.11_Odchudzanie\um0427\FWLib\project/GRAPH.c:337
 134:	9004      	str	r0, [sp, #16]
D:\STM32\Program\1.11_Odchudzanie\um0427\FWLib\project/GRAPH.c:338
 136:	4630      	mov	r0, r6
 138:	f7ff fffe 	bl	0 <__aeabi_fmul>
 13c:	4601      	mov	r1, r0
 13e:	4620      	mov	r0, r4
 140:	f7ff fffe 	bl	0 <__aeabi_fadd>
 144:	f7ff fffe 	bl	0 <__aeabi_f2iz>
D:\STM32\Program\1.11_Odchudzanie\um0427\FWLib\project/GRAPH.c:345
 148:	2103      	movs	r1, #3
D:\STM32\Program\1.11_Odchudzanie\um0427\FWLib\project/GRAPH.c:338
 14a:	9005      	str	r0, [sp, #20]
D:\STM32\Program\1.11_Odchudzanie\um0427\FWLib\project/GRAPH.c:345
 14c:	2201      	movs	r2, #1
 14e:	4668      	mov	r0, sp
 150:	f7ff fffe 	bl	0 <GRAPH_Arrow>
D:\STM32\Program\1.11_Odchudzanie\um0427\FWLib\project/GRAPH.c:362
 154:	b006      	add	sp, #24
 156:	e8bd 8f70 	ldmia.w	sp!, {r4, r5, r6, r8, r9, sl, fp, pc}
 15a:	46c0      	nop			(mov r8, r8)
 15c:	41a00000 	.word	0x41a00000
 160:	41200000 	.word	0x41200000
Disassembly of section .text.GRAPH_Circle:

00000000 <GRAPH_Circle>:
GRAPH_Circle():
D:\STM32\Program\1.11_Odchudzanie\um0427\FWLib\project/GRAPH.c:152
   0:	e92d 4ff0 	stmdb	sp!, {r4, r5, r6, r7, r8, r9, sl, fp, lr}
   4:	461f      	mov	r7, r3
D:\STM32\Program\1.11_Odchudzanie\um0427\FWLib\project/GRAPH.c:156
   6:	ea4f 0342 	mov.w	r3, r2, lsl #1
D:\STM32\Program\1.11_Odchudzanie\um0427\FWLib\project/GRAPH.c:152
   a:	b087      	sub	sp, #28
D:\STM32\Program\1.11_Odchudzanie\um0427\FWLib\project/GRAPH.c:154
   c:	4691      	mov	r9, r2
D:\STM32\Program\1.11_Odchudzanie\um0427\FWLib\project/GRAPH.c:156
   e:	f1c3 0a01 	rsb	sl, r3, #1	; 0x1
  12:	2200      	movs	r2, #0
  14:	2301      	movs	r3, #1
D:\STM32\Program\1.11_Odchudzanie\um0427\FWLib\project/GRAPH.c:152
  16:	9001      	str	r0, [sp, #4]
  18:	468b      	mov	fp, r1
D:\STM32\Program\1.11_Odchudzanie\um0427\FWLib\project/GRAPH.c:156
  1a:	9202      	str	r2, [sp, #8]
  1c:	9303      	str	r3, [sp, #12]
  1e:	9204      	str	r2, [sp, #16]
  20:	9205      	str	r2, [sp, #20]
D:\STM32\Program\1.11_Odchudzanie\um0427\FWLib\project/GRAPH.c:161
  22:	9b05      	ldr	r3, [sp, #20]
  24:	9a01      	ldr	r2, [sp, #4]
  26:	fa5f f689 	uxtb.w	r6, r9
  2a:	eb03 040b 	add.w	r4, r3, fp
  2e:	eb06 0802 	add.w	r8, r6, r2
  32:	fa5f f888 	uxtb.w	r8, r8
  36:	b2e4      	uxtb	r4, r4
  38:	4640      	mov	r0, r8
  3a:	4621      	mov	r1, r4
  3c:	463a      	mov	r2, r7
  3e:	f7ff fffe 	bl	0 <GRAPH_Circle>
D:\STM32\Program\1.11_Odchudzanie\um0427\FWLib\project/GRAPH.c:162
  42:	9a01      	ldr	r2, [sp, #4]
  44:	4621      	mov	r1, r4
  46:	1b95      	subs	r5, r2, r6
  48:	b2ed      	uxtb	r5, r5
  4a:	4628      	mov	r0, r5
  4c:	463a      	mov	r2, r7
  4e:	f7ff fffe 	bl	0 <GRAPH_Circle>
  52:	9b05      	ldr	r3, [sp, #20]
D:\STM32\Program\1.11_Odchudzanie\um0427\FWLib\project/GRAPH.c:163
  54:	4628      	mov	r0, r5
D:\STM32\Program\1.11_Odchudzanie\um0427\FWLib\project/GRAPH.c:162
  56:	ebc3 040b 	rsb	r4, r3, fp
  5a:	b2e4      	uxtb	r4, r4
D:\STM32\Program\1.11_Odchudzanie\um0427\FWLib\project/GRAPH.c:163
  5c:	4621      	mov	r1, r4
  5e:	463a      	mov	r2, r7
  60:	f7ff fffe 	bl	0 <GRAPH_Circle>
D:\STM32\Program\1.11_Odchudzanie\um0427\FWLib\project/GRAPH.c:164
  64:	4640      	mov	r0, r8
  66:	4621      	mov	r1, r4
  68:	463a      	mov	r2, r7
  6a:	f7ff fffe 	bl	0 <GRAPH_Circle>
  6e:	9a05      	ldr	r2, [sp, #20]
  70:	9b01      	ldr	r3, [sp, #4]
D:\STM32\Program\1.11_Odchudzanie\um0427\FWLib\project/GRAPH.c:165
  72:	eb06 050b 	add.w	r5, r6, fp
D:\STM32\Program\1.11_Odchudzanie\um0427\FWLib\project/GRAPH.c:164
  76:	eb02 0803 	add.w	r8, r2, r3
  7a:	fa5f f888 	uxtb.w	r8, r8
D:\STM32\Program\1.11_Odchudzanie\um0427\FWLib\project/GRAPH.c:165
  7e:	b2ed      	uxtb	r5, r5
  80:	4640      	mov	r0, r8
  82:	4629      	mov	r1, r5
  84:	463a      	mov	r2, r7
  86:	f7ff fffe 	bl	0 <GRAPH_Circle>
  8a:	9b05      	ldr	r3, [sp, #20]
  8c:	9a01      	ldr	r2, [sp, #4]
D:\STM32\Program\1.11_Odchudzanie\um0427\FWLib\project/GRAPH.c:167
  8e:	ebc6 060b 	rsb	r6, r6, fp
D:\STM32\Program\1.11_Odchudzanie\um0427\FWLib\project/GRAPH.c:165
  92:	1ad4      	subs	r4, r2, r3
  94:	b2e4      	uxtb	r4, r4
D:\STM32\Program\1.11_Odchudzanie\um0427\FWLib\project/GRAPH.c:166
  96:	4620      	mov	r0, r4
  98:	4629      	mov	r1, r5
  9a:	463a      	mov	r2, r7
D:\STM32\Program\1.11_Odchudzanie\um0427\FWLib\project/GRAPH.c:167
  9c:	b2f6      	uxtb	r6, r6
D:\STM32\Program\1.11_Odchudzanie\um0427\FWLib\project/GRAPH.c:166
  9e:	f7ff fffe 	bl	0 <GRAPH_Circle>
D:\STM32\Program\1.11_Odchudzanie\um0427\FWLib\project/GRAPH.c:167
  a2:	4620      	mov	r0, r4
  a4:	4631      	mov	r1, r6
  a6:	463a      	mov	r2, r7
  a8:	f7ff fffe 	bl	0 <GRAPH_Circle>
D:\STM32\Program\1.11_Odchudzanie\um0427\FWLib\project/GRAPH.c:168
  ac:	463a      	mov	r2, r7
  ae:	4640      	mov	r0, r8
  b0:	4631      	mov	r1, r6
  b2:	f7ff fffe 	bl	0 <GRAPH_Circle>
D:\STM32\Program\1.11_Odchudzanie\um0427\FWLib\project/GRAPH.c:170
  b6:	9a04      	ldr	r2, [sp, #16]
  b8:	9b03      	ldr	r3, [sp, #12]
  ba:	18d2      	adds	r2, r2, r3
D:\STM32\Program\1.11_Odchudzanie\um0427\FWLib\project/GRAPH.c:172
  bc:	eb0a 0342 	add.w	r3, sl, r2, lsl #1
  c0:	2b00      	cmp	r3, #0
D:\STM32\Program\1.11_Odchudzanie\um0427\FWLib\project/GRAPH.c:170
  c2:	9204      	str	r2, [sp, #16]
D:\STM32\Program\1.11_Odchudzanie\um0427\FWLib\project/GRAPH.c:172
  c4:	dd05      	ble.n	d2 <GRAPH_Circle+0xd2>
D:\STM32\Program\1.11_Odchudzanie\um0427\FWLib\project/GRAPH.c:175
  c6:	4452      	add	r2, sl
D:\STM32\Program\1.11_Odchudzanie\um0427\FWLib\project/GRAPH.c:174
  c8:	f109 39ff 	add.w	r9, r9, #4294967295	; 0xffffffff
D:\STM32\Program\1.11_Odchudzanie\um0427\FWLib\project/GRAPH.c:175
  cc:	9204      	str	r2, [sp, #16]
D:\STM32\Program\1.11_Odchudzanie\um0427\FWLib\project/GRAPH.c:176
  ce:	f10a 0a02 	add.w	sl, sl, #2	; 0x2
D:\STM32\Program\1.11_Odchudzanie\um0427\FWLib\project/GRAPH.c:171
  d2:	9a03      	ldr	r2, [sp, #12]
D:\STM32\Program\1.11_Odchudzanie\um0427\FWLib\project/GRAPH.c:169
  d4:	9b02      	ldr	r3, [sp, #8]
D:\STM32\Program\1.11_Odchudzanie\um0427\FWLib\project/GRAPH.c:171
  d6:	3202      	adds	r2, #2
  d8:	9203      	str	r2, [sp, #12]
  da:	9a05      	ldr	r2, [sp, #20]
D:\STM32\Program\1.11_Odchudzanie\um0427\FWLib\project/GRAPH.c:169
  dc:	3301      	adds	r3, #1
  de:	9302      	str	r3, [sp, #8]
D:\STM32\Program\1.11_Odchudzanie\um0427\FWLib\project/GRAPH.c:171
  e0:	1c53      	adds	r3, r2, #1
  e2:	b2db      	uxtb	r3, r3
  e4:	9305      	str	r3, [sp, #20]
D:\STM32\Program\1.11_Odchudzanie\um0427\FWLib\project/GRAPH.c:159
  e6:	9b02      	ldr	r3, [sp, #8]
  e8:	4599      	cmp	r9, r3
  ea:	da9a      	bge.n	22 <GRAPH_Circle+0x22>
D:\STM32\Program\1.11_Odchudzanie\um0427\FWLib\project/GRAPH.c:179
  ec:	b007      	add	sp, #28
  ee:	e8bd 8ff0 	ldmia.w	sp!, {r4, r5, r6, r7, r8, r9, sl, fp, pc}
  f2:	46c0      	nop			(mov r8, r8)
Disassembly of section .text.GRAPH_RectangleFilled:

00000000 <GRAPH_RectangleFilled>:
GRAPH_RectangleFilled():
D:\STM32\Program\1.11_Odchudzanie\um0427\FWLib\project/GRAPH.c:122
   0:	e92d 4ff7 	stmdb	sp!, {r0, r1, r2, r4, r5, r6, r7, r8, r9, sl, fp, lr}
D:\STM32\Program\1.11_Odchudzanie\um0427\FWLib\project/GRAPH.c:134
   4:	2700      	movs	r7, #0
D:\STM32\Program\1.11_Odchudzanie\um0427\FWLib\project/GRAPH.c:122
   6:	9301      	str	r3, [sp, #4]
D:\STM32\Program\1.11_Odchudzanie\um0427\FWLib\project/GRAPH.c:134
   8:	2306      	movs	r3, #6
D:\STM32\Program\1.11_Odchudzanie\um0427\FWLib\project/GRAPH.c:122
   a:	4682      	mov	sl, r0
   c:	4689      	mov	r9, r1
   e:	4616      	mov	r6, r2
  10:	f99d 5030 	ldrsb.w	r5, [sp, #48]
D:\STM32\Program\1.11_Odchudzanie\um0427\FWLib\project/GRAPH.c:134
  14:	fbb2 fbf3 	udiv	fp, r2, r3
  18:	46b8      	mov	r8, r7
D:\STM32\Program\1.11_Odchudzanie\um0427\FWLib\project/GRAPH.c:127
  1a:	e026      	b.n	6a <GRAPH_RectangleFilled+0x6a>
D:\STM32\Program\1.11_Odchudzanie\um0427\FWLib\project/GRAPH.c:128
  1c:	2e05      	cmp	r6, #5
  1e:	d80f      	bhi.n	40 <GRAPH_RectangleFilled+0x40>
  20:	2400      	movs	r4, #0
  22:	e00a      	b.n	3a <GRAPH_RectangleFilled+0x3a>
D:\STM32\Program\1.11_Odchudzanie\um0427\FWLib\project/GRAPH.c:130
  24:	eb04 000a 	add.w	r0, r4, sl
  28:	eb07 0109 	add.w	r1, r7, r9
  2c:	b2c0      	uxtb	r0, r0
  2e:	b2c9      	uxtb	r1, r1
  30:	462a      	mov	r2, r5
  32:	f7ff fffe 	bl	0 <GRAPH_RectangleFilled>
D:\STM32\Program\1.11_Odchudzanie\um0427\FWLib\project/GRAPH.c:129
  36:	1c63      	adds	r3, r4, #1
  38:	b2dc      	uxtb	r4, r3
  3a:	42b4      	cmp	r4, r6
  3c:	d1f2      	bne.n	24 <GRAPH_RectangleFilled+0x24>
  3e:	e010      	b.n	62 <GRAPH_RectangleFilled+0x62>
D:\STM32\Program\1.11_Odchudzanie\um0427\FWLib\project/GRAPH.c:133
  40:	4650      	mov	r0, sl
  42:	eb08 0109 	add.w	r1, r8, r9
  46:	f7ff fffe 	bl	0 <GLCD_GoTo>
  4a:	2400      	movs	r4, #0
D:\STM32\Program\1.11_Odchudzanie\um0427\FWLib\project/GRAPH.c:134
  4c:	e007      	b.n	5e <GRAPH_RectangleFilled+0x5e>
D:\STM32\Program\1.11_Odchudzanie\um0427\FWLib\project/GRAPH.c:135
  4e:	b10d      	cbz	r5, 54 <GRAPH_RectangleFilled+0x54>
D:\STM32\Program\1.11_Odchudzanie\um0427\FWLib\project/GRAPH.c:136
  50:	20ff      	movs	r0, #255
  52:	e000      	b.n	56 <GRAPH_RectangleFilled+0x56>
D:\STM32\Program\1.11_Odchudzanie\um0427\FWLib\project/GRAPH.c:138
  54:	4628      	mov	r0, r5
  56:	f7ff fffe 	bl	0 <GLCD_Write8Pixels>
D:\STM32\Program\1.11_Odchudzanie\um0427\FWLib\project/GRAPH.c:134
  5a:	1c63      	adds	r3, r4, #1
  5c:	b2dc      	uxtb	r4, r3
  5e:	455c      	cmp	r4, fp
  60:	d1f5      	bne.n	4e <GLCD_Write8Pixels+0x4e>
D:\STM32\Program\1.11_Odchudzanie\um0427\FWLib\project/GRAPH.c:127
  62:	1c7b      	adds	r3, r7, #1
  64:	b2df      	uxtb	r7, r3
  66:	f108 0801 	add.w	r8, r8, #1	; 0x1
  6a:	9b01      	ldr	r3, [sp, #4]
  6c:	429f      	cmp	r7, r3
  6e:	d1d5      	bne.n	1c <GLCD_Write8Pixels+0x1c>
D:\STM32\Program\1.11_Odchudzanie\um0427\FWLib\project/GRAPH.c:146
  70:	e8bd 8ffe 	ldmia.w	sp!, {r1, r2, r3, r4, r5, r6, r7, r8, r9, sl, fp, pc}
Disassembly of section .text.GRAPH_WriteChar:

00000000 <GRAPH_WriteChar>:
GRAPH_WriteChar():
D:\STM32\Program\1.11_Odchudzanie\um0427\FWLib\project/GRAPH.c:57
   0:	280c      	cmp	r0, #12
D:\STM32\Program\1.11_Odchudzanie\um0427\FWLib\project/GRAPH.c:54
   2:	b537      	push	{r0, r1, r2, r4, r5, lr}
   4:	4605      	mov	r5, r0
D:\STM32\Program\1.11_Odchudzanie\um0427\FWLib\project/GRAPH.c:57
   6:	d004      	beq.n	12 <GRAPH_WriteChar+0x12>
   8:	280d      	cmp	r0, #13
   a:	d013      	beq.n	34 <GRAPH_WriteChar+0x34>
   c:	280a      	cmp	r0, #10
   e:	d008      	beq.n	22 <GRAPH_WriteChar+0x22>
  10:	e015      	b.n	3e <GRAPH_WriteChar+0x3e>
D:\STM32\Program\1.11_Odchudzanie\um0427\FWLib\project/GRAPH.c:59
  12:	f7ff fffe 	bl	0 <GRAPH_WriteChar>
D:\STM32\Program\1.11_Odchudzanie\um0427\FWLib\project/GRAPH.c:60
  16:	4b24      	ldr	r3, [pc, #144]	(a8 <GRAPH_WriteChar+0xa8>)
  18:	2000      	movs	r0, #0
  1a:	7058      	strb	r0, [r3, #1]
D:\STM32\Program\1.11_Odchudzanie\um0427\FWLib\project/GRAPH.c:61
  1c:	7018      	strb	r0, [r3, #0]
D:\STM32\Program\1.11_Odchudzanie\um0427\FWLib\project/GRAPH.c:62
  1e:	4601      	mov	r1, r0
  20:	e005      	b.n	2e <GRAPH_WriteChar+0x2e>
D:\STM32\Program\1.11_Odchudzanie\um0427\FWLib\project/GRAPH.c:66
  22:	4b21      	ldr	r3, [pc, #132]	(a8 <GRAPH_WriteChar+0xa8>)
  24:	7859      	ldrb	r1, [r3, #1]
D:\STM32\Program\1.11_Odchudzanie\um0427\FWLib\project/GRAPH.c:67
  26:	7818      	ldrb	r0, [r3, #0]
D:\STM32\Program\1.11_Odchudzanie\um0427\FWLib\project/GRAPH.c:66
  28:	3101      	adds	r1, #1
  2a:	b2c9      	uxtb	r1, r1
  2c:	7059      	strb	r1, [r3, #1]
D:\STM32\Program\1.11_Odchudzanie\um0427\FWLib\project/GRAPH.c:67
  2e:	f7ff fffe 	bl	0 <GRAPH_WriteChar>
D:\STM32\Program\1.11_Odchudzanie\um0427\FWLib\project/GRAPH.c:68
  32:	e037      	b.n	a4 <GRAPH_WriteChar+0xa4>
D:\STM32\Program\1.11_Odchudzanie\um0427\FWLib\project/GRAPH.c:71
  34:	4b1c      	ldr	r3, [pc, #112]	(a8 <GRAPH_WriteChar+0xa8>)
  36:	2000      	movs	r0, #0
  38:	7018      	strb	r0, [r3, #0]
D:\STM32\Program\1.11_Odchudzanie\um0427\FWLib\project/GRAPH.c:72
  3a:	7859      	ldrb	r1, [r3, #1]
  3c:	e7f7      	b.n	2e <GRAPH_WriteChar+0x2e>
D:\STM32\Program\1.11_Odchudzanie\um0427\FWLib\project/GRAPH.c:77
  3e:	4b1b      	ldr	r3, [pc, #108]	(ac <GRAPH_WriteChar+0xac>)
  40:	4c19      	ldr	r4, [pc, #100]	(a8 <GRAPH_WriteChar+0xa8>)
  42:	781b      	ldrb	r3, [r3, #0]
  44:	2bff      	cmp	r3, #255
  46:	d110      	bne.n	6a <GRAPH_WriteChar+0x6a>
D:\STM32\Program\1.11_Odchudzanie\um0427\FWLib\project/GRAPH.c:79
  48:	2081      	movs	r0, #129
  4a:	f7ff fffe 	bl	0 <GLCD_Write_Command>
D:\STM32\Program\1.11_Odchudzanie\um0427\FWLib\project/GRAPH.c:80
  4e:	7820      	ldrb	r0, [r4, #0]
  50:	2206      	movs	r2, #6
  52:	fb00 f002 	mul.w	r0, r0, r2
  56:	7861      	ldrb	r1, [r4, #1]
  58:	2301      	movs	r3, #1
  5a:	00c9      	lsls	r1, r1, #3
  5c:	9300      	str	r3, [sp, #0]
  5e:	f000 00fe 	and.w	r0, r0, #254	; 0xfe
  62:	f001 01f8 	and.w	r1, r1, #248	; 0xf8
  66:	3307      	adds	r3, #7
  68:	e00f      	b.n	8a <GRAPH_WriteChar+0x8a>
D:\STM32\Program\1.11_Odchudzanie\um0427\FWLib\project/GRAPH.c:85
  6a:	2080      	movs	r0, #128
  6c:	f7ff fffe 	bl	0 <GLCD_Write_Command>
D:\STM32\Program\1.11_Odchudzanie\um0427\FWLib\project/GRAPH.c:86
  70:	7820      	ldrb	r0, [r4, #0]
  72:	2206      	movs	r2, #6
  74:	fb00 f002 	mul.w	r0, r0, r2
  78:	7861      	ldrb	r1, [r4, #1]
  7a:	2300      	movs	r3, #0
  7c:	00c9      	lsls	r1, r1, #3
  7e:	9300      	str	r3, [sp, #0]
  80:	f000 00fe 	and.w	r0, r0, #254	; 0xfe
  84:	f001 01f8 	and.w	r1, r1, #248	; 0xf8
  88:	3308      	adds	r3, #8
  8a:	f7ff fffe 	bl	0 <GRAPH_WriteChar>
D:\STM32\Program\1.11_Odchudzanie\um0427\FWLib\project/GRAPH.c:87
  8e:	7820      	ldrb	r0, [r4, #0]
  90:	7861      	ldrb	r1, [r4, #1]
  92:	f7ff fffe 	bl	0 <GRAPH_WriteChar>
D:\STM32\Program\1.11_Odchudzanie\um0427\FWLib\project/GRAPH.c:88
  96:	4628      	mov	r0, r5
  98:	f7ff fffe 	bl	0 <GLCD_Write_Char>
D:\STM32\Program\1.11_Odchudzanie\um0427\FWLib\project/GRAPH.c:91
  9c:	4a02      	ldr	r2, [pc, #8]	(a8 <GRAPH_WriteChar+0xa8>)
  9e:	7813      	ldrb	r3, [r2, #0]
  a0:	3301      	adds	r3, #1
  a2:	7013      	strb	r3, [r2, #0]
D:\STM32\Program\1.11_Odchudzanie\um0427\FWLib\project/GRAPH.c:94
  a4:	bd3e      	pop	{r1, r2, r3, r4, r5, pc}
  a6:	46c0      	nop			(mov r8, r8)
	...
Disassembly of section .text.GRAPH_Rectangle:

00000000 <GRAPH_Rectangle>:
GRAPH_Rectangle():
D:\STM32\Program\1.11_Odchudzanie\um0427\FWLib\project/GRAPH.c:107
   0:	e92d 47f0 	stmdb	sp!, {r4, r5, r6, r7, r8, r9, sl, lr}
   4:	4680      	mov	r8, r0
   6:	460f      	mov	r7, r1
   8:	4692      	mov	sl, r2
   a:	4699      	mov	r9, r3
   c:	f99d 6020 	ldrsb.w	r6, [sp, #32]
  10:	2500      	movs	r5, #0
D:\STM32\Program\1.11_Odchudzanie\um0427\FWLib\project/GRAPH.c:110
  12:	e010      	b.n	36 <GRAPH_Rectangle+0x36>
  14:	19ec      	adds	r4, r5, r7
  16:	b2e4      	uxtb	r4, r4
D:\STM32\Program\1.11_Odchudzanie\um0427\FWLib\project/GRAPH.c:111
  18:	4640      	mov	r0, r8
  1a:	4621      	mov	r1, r4
  1c:	4632      	mov	r2, r6
  1e:	f7ff fffe 	bl	0 <GRAPH_Rectangle>
D:\STM32\Program\1.11_Odchudzanie\um0427\FWLib\project/GRAPH.c:112
  22:	f108 30ff 	add.w	r0, r8, #4294967295	; 0xffffffff
  26:	4450      	add	r0, sl
  28:	b2c0      	uxtb	r0, r0
  2a:	4621      	mov	r1, r4
  2c:	4632      	mov	r2, r6
  2e:	f7ff fffe 	bl	0 <GRAPH_Rectangle>
D:\STM32\Program\1.11_Odchudzanie\um0427\FWLib\project/GRAPH.c:110
  32:	1c6b      	adds	r3, r5, #1
  34:	b2dd      	uxtb	r5, r3
  36:	454d      	cmp	r5, r9
  38:	d1ec      	bne.n	14 <GRAPH_Rectangle+0x14>
  3a:	2500      	movs	r5, #0
  3c:	e010      	b.n	60 <GRAPH_Rectangle+0x60>
  3e:	eb05 0408 	add.w	r4, r5, r8
  42:	b2e4      	uxtb	r4, r4
D:\STM32\Program\1.11_Odchudzanie\um0427\FWLib\project/GRAPH.c:116
  44:	4620      	mov	r0, r4
  46:	4639      	mov	r1, r7
  48:	4632      	mov	r2, r6
  4a:	f7ff fffe 	bl	0 <GRAPH_Rectangle>
D:\STM32\Program\1.11_Odchudzanie\um0427\FWLib\project/GRAPH.c:117
  4e:	1e79      	subs	r1, r7, #1
  50:	4449      	add	r1, r9
  52:	4620      	mov	r0, r4
  54:	b2c9      	uxtb	r1, r1
  56:	4632      	mov	r2, r6
  58:	f7ff fffe 	bl	0 <GRAPH_Rectangle>
D:\STM32\Program\1.11_Odchudzanie\um0427\FWLib\project/GRAPH.c:115
  5c:	1c6b      	adds	r3, r5, #1
  5e:	b2dd      	uxtb	r5, r3
  60:	4555      	cmp	r5, sl
  62:	d1ec      	bne.n	3e <GRAPH_Rectangle+0x3e>
D:\STM32\Program\1.11_Odchudzanie\um0427\FWLib\project/GRAPH.c:119
  64:	e8bd 87f0 	ldmia.w	sp!, {r4, r5, r6, r7, r8, r9, sl, pc}
